:020000040000FA
:040000001FEF00F0FE
:08000800036A026EFF0E0226DE
:10001000032200D0D8A01200030E016EE70E02D812
:10002000F5D7016AFD0F006EFF0E00D001D000264B
:10003000000000D0D8A00126D8A01200F8D7F86A96
:10004000AB6A400EAF6E900EAB6E200EAC6E0B0E18
:10005000C16EF19E096A086A320E0A6EC80E066EFB
:100060000A0E076E5BEC00F094928292320ECCDFA7
:1000700094928282320EC8DF80BA41EF00F09498E9
:10008000829880AA46EF00F09498828881B64BEF60
:1000900000F0949A829A81A650EF00F0949A828A96
:1000A00081B855EF00F09390819081A85AEF00F04D
:1000B00093908180D9D794988298949A829A9390B9
:0C00C0008190939281929394819412009D
:020000040030CA
:03000100061F1FB8
:020005008385F1
:060008000FC00FE00F40E5
:00000001FF
